:1000000000308A001A280000223084008313000880
:10001000031917280230F800F701F70B0D28F80B29
:100020000C289730F700F70B1328800B0A288A1149
:100030000A123D2803081F398300713083168F0090
:1000400090010F0803170908C039890003131F1214
:100050009F120030031788008312870188018901ED
:1000600083130030831603138500850183128501F5
:100070000230A100FA30A2000428A10B3A2883160E
:0C0080000510013083128506382863004B
:04400E00E420FF3F6C
:00000001FF
;PIC16F886
;CRC=B12F  CREATED="18-oct.-22 17:03"
